:020000040800F2
:10000000181C00207902000821300008712E000819
:100010001D300008B5040008F5500008000000007D
:100020000000000000000000000000005D3100083A
:10003000610500080000000025300008613100085B
:10004000930200089302000893020008930200083C
:10005000930200089302000893020008930200082C
:10006000930200089302000893020008930200081C
:10007000930200089302000893020008930200080C
:1000800093020008930200089302000893020008FC
:1000900093020008930200089302000893020008EC
:1000A00093020008930200089302000893020008DC
:1000B0009302000800000000000000009302000806
:1000C00093020008930200089302000893020008BC
:1000D00093020008930200089302000893020008AC
:1000E00093020008930200080000000000000000D6
:1000F0000000000000000000000000000000000000
:1001000000000000930200080000000093020008B5
:1001100000000000000000009302000893020008A5
:10012000930200089302000893020008930200085B
:100130009302000800000000000000000000000022
:10014000930200089302000893020008914F0008F0
:10015000930200089302000893020008930200082B
:1001600093020008930200089302000800000000B8
:1001700093020008930200089302000800000000A8
:1001800093020008930200089302000800F002F8AE
:1001900000F062F814A696E8000CB244B344DA45C5
:1001A00001D100F059F8BAE80F000FA696E8300028
:1001B000A5EB040504EB0607AAEB0704A7F101076A
:1001C0004FEA15154FEA3414A4F10104AC4201D3EF
:1001D00000F042F813F0010F18BFFB1A43F00103BF
:1001E00000F001F8DBE71847505C0000705C00008D
:1001F0000A4410F8014B14F00F0508BF10F8015B1A
:10020000240908BF10F8014B6D1E05D010F8013B02
:100210006D1E01F8013BF9D1641E03D0641E01F884
:10022000015BFBD19142E4D37047000070470000AE
:100230000023002400250026103A28BF78C1FBD8EF
:10024000520728BF30C148BF0B6070471FB505F08B
:10025000C1FC1FBD10B510BD00F0F1F81146FFF74D
:10026000F5FF04F0ABFF00F00FF903B4FFF7F2FF66
:1002700003BC00F017F9000009488047094800470F
:10028000FEE7FEE7FEE7FEE7FEE7FEE7FEE7FEE746
:10029000FEE7FEE704480549054A064B70470000A3
:1002A000E93100088D01000818160020181C0020F4
:1002B0001818002018180020032A40F2308010F08F
:1002C000030C00F0158011F8013BBCF1020F6244F1
:1002D00098BF11F801CB00F8013B38BF11F8013B82
:1002E000A2F1040298BF00F801CB38BF00F8013B2F
:1002F00011F0030300F07180083AC0F0088051F853
:10030000043B083A51F804CBA0E80810F5E7121DA9
:100310005CBF51F8043B40F8043BAFF30080D207C8
:1003200024BF11F8013B11F801CB48BF11F8012B94
:1003300024BF00F8013B00F801CB48BF00F8012BB7
:1003400070474FF000020429C0F0128010F0030C37
:1003500000F01B80CCF1040CBCF1020F18BF00F8B8
:10036000012BA8BF20F8022BA1EB0C0100F00DB867
:100370005FEAC17C24BF00F8012B00F8012B48BFC5
:1003800000F8012B70474FF0000200B51346944669
:100390009646203922BFA0E80C50A0E80C50B1F1DD
:1003A0002001BFF4F7AF090728BFA0E80C5048BFF1
:1003B0000CC05DF804EB890028BF40F8042B08BF8F
:1003C000704748BF20F8022B11F0804F18BF00F88B
:1003D000012B704770477047704710B5203AC0F046
:1003E0000B80B1E81850A0E81850B1E81850A0E808
:1003F0001850203ABFF4F5AF5FEA027C24BFB1E8A1
:100400001850A0E8185044BF18C918C0BDE81040E3
:100410005FEA827C24BF51F8043B40F8043B08BFEC
:100420007047D20728BF31F8023B48BF11F8012BB3
:1004300028BF20F8023B48BF00F8012B70477546E3
:1004400000F02CF8AE4605006946534620F0070040
:10045000854618B020B5FFF71DFFBDE820404FF0DE
:1004600000064FF000074FF000084FF0000BAC46BD
:10047000ACE8C009ACE8C009ACE8C009ACE8C00908
:1004800021F007018D46704710B50446AFF3008098
:100490002046BDE81040FFF7E8BE00000048704766
:1004A0004801002001491820ABBEFEE726000200EB
:1004B00070470000FEE700000020704700207047F2
:1004C00010B540F6F054C2F2000440F6DC11C2F25E
:1004D00000012046002203F053F840F2DC51C2F242
:1004E0000001204603F03EF8002010BD70B540F634
:1004F000F0560546C2F200060C463046294603F087
:1005000031F8304603F008F8206840B1002600BFFB
:10051000A85D05F0DBF9206801368642F8D300209B
:1005200070BD00000020704740F6F052C2F2000299
:10053000D2F8BC22D2F81432002B1CBF0120704725
:1005400010B540F6F054C2F200040A4601462046B7
:1005500003F016F82046BDE8104003F089B800000B
:1005600070470000EFF3108072B600BFFEE7000096
:1005700080B586B00022CDE90122CDE903200591A6
:10058000EFF3108072B602A801A900F06FF90028FD
:1005900018BF4FF0FF3062B606B080BD40F21C10AD
:1005A000C2F20000027F02F0FD01012942F20001C7
:1005B000C4F202010FD10B6823F400730B600B68C7
:1005C00043F400630B600B6823F400630B600B685B
:1005D00043F400730B6002F0FE02022A0BD10A689A
:1005E00042F480520A600A6822F480520A600A6863
:1005F00042F480620A6000210177704753071CBFF4
:100600004FF0FF307047002A04BF00207047B0B59C
:100610004FEAD20C00224FF0000E00BF00EBC203E5
:10062000D3E9003401EBC20541F832304EF001024B
:1006300092B294456C602AD900EBC203D3E900342E
:1006400001EBC20541F832304EF0020292B29445FD
:100650006C601CD900EBC203D3E9003401EBC20586
:1006600041F832304EF0030292B294456C600ED9DC
:1006700000EBC203D3E900340EF1040E01EBC20516
:1006800041F832301FFA8EF294456C60C6D80020D3
:10069000B0BD0000F0B581B042F210060446C4F2CD
:1006A000020600F06FFB3168C9030FD430684CF2CA
:1006B000FA31C0F20201014019D040F21C10C2F21E
:1006C000000042680A434260012016E00546671CAC
:1006D00003E000BF3068C003E8D5002FFAD000F077
:1006E00051FB401BA042F5D3032001B0F0BD3068A0
:1006F000C0074FF0000001D00121316001B0F0BD12
:1007000070B582B014460D46019000F041FA14B362
:100710004FF6FD76C0F603060198B0421BD8EFF302
:10072000108072B60199D5E90023002000F050F93D
:1007300062B6E0B90198D5E90023D0E9000159403B
:100740005040084313D10198013C00F1080005F125
:1007500008050190E0D162B600F030F9019840F64A
:10076000E851C2F200010860002002B070BD00F044
:1007700025F94FF0FF3002B070BD000079B1F0B53F
:1007800045F6384345F6385E01F0030C0429C0F6FF
:100790000003C0F6000E05D2FF22FF212BE0FF214F
:1007A000FF224AE021F003040025FF22FF2100BFC1
:1007B00010F8046BD2B272409E5C10F8037CC9B290
:1007C000714079401EF802205E5C10F8027C724095
:1007D0007A401EF801109E5C10F8017C714079404F
:1007E0001EF802205E5C04351EF80110AFB2A7426D
:1007F00082EA0602DCD1BCF1000F1CD00478D2B230
:1008000054401A5DBCF1010F82EA01021EF8041087
:1008100011D04478D2B254401A5DBCF1020F82EA82
:1008200001021EF8041006D08078D2B250401A5C43
:100830004A401EF80010BDE8F040D0B240EA012066
:1008400080B27047B0B5044600F09CFA054640F20D
:100850003D10C2F200000078611C18BF044400BFC4
:1008600000F090FA401BA042FAD3B0BD2DE9F0474A
:1008700040F21C19C2F2000999F80020012A04BFB5
:100880000220BDE8F0870546012089F800004CF2FF
:1008900050308846FFF7FEFE002840F08A8042F282
:1008A00000070020C4F20207C9F80400386839685C
:1008B000490502D4C0F3402009E0396810F4007003
:1008C0004FF0030021F4806108BF0220396089F8ED
:1008D0001C002868012813D12879C00703D0786943
:1008E00040F004007861786940F4803078614CF21F
:1008F0005030FFF7CFFE796921F0040179612FE0D4
:100900004FF0FF30C8F80000D5E90240204484428F
:1009100022D2E60040F2FA3A786906F4FF6120F448
:100920007E7008437861786940F0020078617869E8
:1009300040F4803078614CF25030FFF7ABFE7969BB
:1009400021EA0A01796148B9D5E902010134084474
:10095000844206F10806DFD3002001E0C8F8004019
:1009600099F81C1001F0FD02012A0FD13A6822F417
:1009700000723A603A6842F400623A603A6822F4DF
:1009800000623A603A6842F400723A6001F0FE0197
:1009900002290BD1396841F480513960396821F45A
:1009A00080513960396841F480613960002189F8EB
:1009B0001C10002189F80010BDE8F08742F21401F4
:1009C000C4F20201086840F0004200200A6070474B
:1009D0002DE9F04F81B040F21C1AC2F2000A9AF8D9
:1009E0000070012F03D1022001B000F0CDB8054600
:1009F00042F21006012099468B469046C4F2020648
:100A00008AF8000000F0BEF93168C9030AD504462F
:100A10004CF24F3700F0B6F9001BB8426BD8306883
:100A2000C003F7D430684CF2FA31C0F2020108403A
:100A300007D0DAF804100143CAF80410306001202E
:100A40009CE030680021C0071CBF01203060CAF85C
:100A5000041056F8100C4005284606D556F8101C10
:100A600021F4806146F8101C022100288AF81C102D
:100A700043D002284FD87168A8F1400341F4802187
:100A80007160EFF31081EFF3108272B6ABF14002A8
:100A9000402700BF53F8405F103F42F8405F5D6859
:100AA0003C0655609D689560DD68D5601D691561DF
:100AB0005D6955619D699561DD69D5611D6A156244
:100AC0005D6A55629D6A9562DD6AD5621D6B15632C
:100AD0005D6B55639D6B9563DD6BD563DAD1871EC6
:100AE00018BF012781F310886FF48029022818BFEE
:100AF0004FF0FF3912E0032040E07068002740F01B
:100B000001007060CBF80080BFF36F8FCBF80490CA
:100B10006FF0010902E04FF0FF39012700F032F9D0
:100B20003168C9030AD504464CF24F3500F02AF962
:100B3000001BA84218D83068C003F7D430684CF2C4
:100B4000FA31C0F20201014006D0DAF8040008438D
:100B5000CAF80400012005E03068C0074FF000002B
:100B600003D00121316000E0032004461FB9706802
:100B700000EA09007060FFF711FD204600218AF8A5
:100B8000001001B000F000B830BCBDE8C08F00001C
:100B900042F20800C4F20200C168B1F1FF3FC4BFD5
:100BA0000020704740F22311C4F26751016048F6FB
:100BB000AB11CCF6EF510160C068C00F7047000068
:100BC0002DE9F04F83B00E68002E00F0CE8000F1CA
:100BD000200241F2000C009200F13847C4F6000CEC
:100BE00007224FEAB725604508BF0422042D38BF0D
:100BF0004FEAB722002500274FF0000801920AE0D3
:100C00000E6808F1010836FA08F207F1020705F14B
:100C1000040500F0AA80012202FA08FE16EA0E0975
:100C2000EED0D1F804C003220CF0030BABF10106A7
:100C300002FA07F4012E6FEA040A11D88468CE681C
:100C400004EA0A04BE4034438460446824EA0E0681
:100C5000CCF3001404FA08F42643466006E000BF13
:100C6000BBF1030F02D14FF0030B21E0C6688C6883
:100C700006EA0A06BC402643BBF1020FC66017D144
:100C80006FF00302009B02EA580605F01C020F24D5
:100C900053F806C004FA02FE0C692CEA0E0C04FAA2
:100CA00002F242EA0C029A51D1F804C00CF0030B94
:100CB00002680BFA07F302EA0A021A431CF4403FE7
:100CC00002609DD041F26003C4F202031A6840F250
:100CD000004E42F001021A601A68C4F2010E02F0DE
:100CE00001020292029A28F003024FF6084C724465
:100CF000CFF6FF7C52F80C3005F00C060F24B44000
:100D0000A343019C04FA06F6334342F80C30DEF8A4
:100D100008204B6842EA090640F20C4CDC0258BF3E
:100D200022EA0906CEF80860C4F2010CDCF80020C3
:100D30009C0242EA090658BF22EA0906CCF8006084
:100D4000DEF804209C0342EA090658BF22EA09069D
:100D5000CEF80460DEF80020DB0342EA090658BF43
:100D600022EA0906CEF800604AE703B000F000B8B6
:100D700030BCBDE8C08F00001823002A08BF28231C
:100D8000C150704741F21460C2F200000068704721
:100D900040F23D1041F21461C2F20000C2F20001C3
:100DA00000780A68104408607047000080B503208E
:100DB00000F0A8F80F2000F009F800281CBF01205F
:100DC00080BD00F031F8002080BD000040F23D11F0
:100DD000C2F200010978002904BF0120704710B554
:100DE000044640F22400C2F200004FF47A72006818
:100DF000B2FBF1F1B0FBF1F002F024F801460F2C48
:100E00004FF001000ED8002918BF10BD4FF0FF3081
:100E10002146002200F04AF840F240110020C2F2C0
:100E200000010C6010BD000082B041F25800C4F215
:100E30000200816841F001018160816801F00101D7
:100E400001910199016841F080510160006800F052
:100E500080500090009802B070470000002848BF02
:100E6000704700F01F01012202FA01F11C2202EA80
:100E7000D0004EF28012CEF200028150BFF34F8FAD
:100E8000BFF36F8F70470000002848BF704700F025
:100E90001F01012202FA01F11C2202EAD0004EF2E7
:100EA0000012CEF2000281507047000010B54EF6DD
:100EB0000C5CCEF2000CDCF80030C3F3022E8EF096
:100EC0000704042C28BF0424BEF103034FF0FF3EA7
:100ED0000EFA04F438BF0023A14399400EFA03F33D
:100EE0009A43114300F00F0200F160430901043AF4
:100EF00003F564436244002848BF02F10C031970F3
:100F000010BD00004EF60C51CEF200010A684FF6FB
:100F1000FF031A4060F30A2242F0806040F0FD7047
:100F20000860704704F0E8F801220168C0F8D42294
:100F3000002280F8C822B1F8540040F00100A1F866
:100F40005400B1F8540040F002020020A1F85420EF
:100F50007047000010B50129044612D009BBA07AE1
:100F600048B102F0FFF84EF61050CEF200000168D2
:100F700021F006010160D4F8DC02BDE8104002F067
:100F8000F5BED4F8DC0202F087FFA07A002808BF83
:100F900010BD4EF61050CEF20000016841F006017F
:100FA000016010BD80B501F0070C0CEB8C0C00EB60
:100FB000CC0C0CF1100C01EB810E090600EBCE00FD
:100FC00058BF00F5A87C2AB1ACF808301B0C0121F1
:100FD0000A2001E0002106202CF8003000208CF8C7
:100FE0000C1080BD01EB8102D0F8DC3200EBC200B6
:100FF000426A184602F060BD01EB8102D0F8DC3293
:1010000000EBC200D0F86421184602F0AFBD00002A
:10101000002804BF0120704710B50446032084F85F
:101020009102206804F010F800281CBF012010BDB8
:10103000204600F079FE002084F8910210BD0000E7
:1010400010B54FFA81FC4FF4A87201F0070EBCF105
:10105000000F48BF102290F8904202440EEB8E031E
:101060004FEAD11C02EBC301012C81F801C002F848
:1010700033E004BF022010BD0268012380F89032E3
:101080000446104603F05EFB002084F8900210BD79
:10109000B0B5027901F00F03934284BF0120B0BDC7
:1010A0004AB24FF4A874002A48BF102401F0070E7A
:1010B000021990F890420EEB8E034FEAD11C02EB1E
:1010C000C301012C4FF0000481F801C08C7002F8BC
:1010D00033E004BF0220B0BD0268012380F89032E3
:1010E0000546104603F0CAFB204685F89042B0BD85
:1010F00001F0070101EB810100EBC100D0F86C01A8
:1011000070470000B0B54FFA81FC4FF4A87401F0AD
:10111000070EBCF1000F48BF102404440EEB8E05EF
:101120004FEAD11C04EBC5016FF3DF2281F801C047
:1011300004F835E00A61022BCB7004BF00220A716B
:1011400090F89022012A04BF0220B0BD026801235A
:1011500080F890320446104603F072F9002084F8BB
:101160009002B0BD10B501F0070C0CEB8C0100EB48
:10117000C10E00680EF5A8710024CEF86421CEF8E7
:101180006831CEF86C418EF851418EF850C103F0B1
:10119000C5FB002010BD0000B0B5027901F00704C6
:1011A00094424FF001022BD84BB24FF4A875002B9C
:1011B00048BF10254FEAD11C48BF2146054401EB2A
:1011C000810305EBC30181F801C090F890C28A70D9
:1011D000BCF1010F05F8334004BF0220B0BD026826
:1011E0000123054680F89032104603F07DFB24B9B8
:1011F000286805F5267103F03FFB002285F8902250
:101200001046B0BD80B501F0070C0CEB8C0100EB73
:10121000C10101F810CF00684FF0010C01F1140773
:1012200081F824C04FF0000E87E80C400B6281F873
:1012300001C003F073FB002080BD00002DE9F04FDA
:1012400083B00446006803F0A9FE01041DD44105E3
:1012500000F18F83410400F19D83810400F1AE838E
:10126000C10400F1B183010500F1D383010600F14F
:10127000E583810500F1F283C00540F18883206891
:10128000B0F8441021F48071BEE32068B0F9441036
:10129000B1F1FF3F00F37B8304F5A871019104F1E4
:1012A000100148F2C005029104F5267140F60F784E
:1012B000009122E0B0F8501094F85021014401EB65
:1012C000C201B1F80634B4F8562100996FF39F2398
:1012D000C4F86C3103F066FE2068018801EA080159
:1012E00080310180204600F0B5FD00BF2068B0F9D4
:1012F0004410B1F1FF3F00F34A83B0F8442012F0EC
:101300000F090DD030F929104FEA490BB1F1FF3F19
:101310001FFA81FA2EDD5FEA0A60E7D52AE100BFF5
:101320000188D2065DD401EA080101F5004101807F
:10133000B0F85010227C084400EBC200B0F8020460
:10134000616A6FF39F20E0620844606220460021DA
:10135000FFF748FE607B0028C8D0A06A0028C5D1EE
:10136000607B216840F08000C0B2A1F84C000020F2
:101370006073BBE730F81B1001EA0801803120F8E8
:101380001B10019A09EB890102EBC106317B002990
:101390006AD0F178022976D1B0F850303178B2694C
:1013A00003445FEA4A4703EBC10300F18380B3F8CB
:1013B000067400236FF39F27D21B38BF1A46B26111
:1013C00040F28D805FEA4A6200F1978030F8212078
:1013D00002EA08022A4320F82120002F40F08E80E4
:1013E000AAE00A053FF566AF09B2B1F1FF3F3FF74A
:1013F0007DAF018801EA080180310180B0F850100A
:1014000094F85021014401EBC201B1F806346FF3A6
:101410009F23C4F86C3193B1D4F8641179B1B4F856
:10142000562103F0BFFDD4F86401D4F86C110844D0
:10143000C4F8640120460021FFF7DEFD2068018822
:101440000A053FF553AF01F44051B1F5405F3FF459
:101450004DAF018843F60F7211404CF28002A2F5A5
:1014600080525140018041E7B0F850103278014479
:1014700001EBC201B1F806746FF39F27002F5BD018
:101480007169F28854E0317830F8212002EA0802CC
:101490002A4320F8212030F82120B0F8503000EB0A
:1014A000C1015204194414D4B1F806746FF39F2794
:1014B00027BB41E0B3F8027400236FF39F27D21BD0
:1014C00038BF1A46B2611CD95FEA4A6226D46FBBA4
:1014D00032E0B1F802746FF39F273FBB2CE030F885
:1014E000212043F60F731A4005F5FE535A4020F8A9
:1014F00021205FEA4A627FF569AFEFB171697289B5
:1015000016E030F8212043F60F731A4005F5FE531C
:101510005A4020F821205FEA4A62D8D530F82120CD
:1015200002EA08022A4320F821202FB1716932898A
:101530003B4603F037FD00E00027F169D6E90502DC
:1015400039443844F161706112B13069B84208D948
:1015500031782046FFF750FD5FEA0A607FF5C6AE9E
:1015600008E02068314603F0D9F95FEA0A607FF5A8
:10157000BDAE00BF206809EB890130F81B20029B3B
:1015800003EBC10602EA080101F5004120F81B1037
:10159000F378012B21D1317B00294FF00001B1619B
:1015A00000F01A815FEA4A6171D47178012900F074
:1015B0000081002940F01081B0F8501032780844C2
:1015C00000EBC200B0F806146FF39F21A0F80614D8
:1015D000B0F8061441F40041F2E05FEACA511CD4AD
:1015E000B0F850203178024402EBC102B2F8022474
:1015F000B3696FF39F229B1A4FF0000738BF3B4639
:10160000B36140F2EA807169F3691144716199181C
:10161000F161314603F082F968E6B0F85050317854
:10162000B2695FEA4A6700EBC10E48D40EF2064C7D
:101630003CF8055000276FF39F25521B38BF3A46F0
:10164000B2616CD95FEA4A4208D430F821204CF2EA
:10165000800302EA08021A4320F8212096F8241099
:10166000012940F07781D6E90431D6E9077229448F
:101670002F449A427161F76180F0FB80002A00F0EC
:101680001C810023336286F82430134619E17178F7
:10169000012900F09880002940F09E80B0F8501099
:1016A0003278084400EBC200B0F802146FF39F21B7
:1016B000A0F80214B0F8021441F400418AE00EF2DE
:1016C000024C3CF8055000276FF39F25521B38BF92
:1016D0003A46B26146D95FEA4A4208D530F821203D
:1016E0004CF2800302EA08021A4320F8212096F8FF
:1016F0002410012940F02E81D6E90431D6E90727CC
:1017000029442A449F427161F26180F0B580002231
:10171000002F86F8242040F0B1802F46AFE0727889
:10172000012A5ED0002A48F2C00565D1B0F85020E9
:101730007244B2F802746FF39F27A2F80274B2F8F1
:10174000027447F40047A2F80274B0F850203CF845
:1017500002706FF39F272CF802703CF8027047F478
:10176000004747E07278012A5AD0002A48F2C005A3
:1017700062D1B0F850203CF802506FF39F252CF84E
:1017800002503CF8025045F400452CF80250B0F8E5
:10179000502048F2C0057244B2F806746FF39F27D8
:1017A000A2F80674B2F8067447F40047A2F806746B
:1017B00042E0B0F850103278084400EBC20000213B
:1017C000A0F8061408E0B0F850103278084400EB96
:1017D000C2000021A0F8021431782046FFF702FC75
:1017E00084E5B0F8502048F2C0057244A2F80274B3
:1017F000B0F850202CF80270022B09D130F82120CB
:1018000040F63F731A40A5F120035A4020F82120EA
:101810002046FFF7E7FB5FEA4A403FF567AD1EE071
:10182000B0F8502000252CF80250B0F85020724437
:10183000A2F8065448F2C005022B09D130F8212045
:1018400040F63F731A40A5F120035A4020F82120AA
:101850002046FFF7C7FB5FEA4A407FF547AD2068A7
:1018600031784CF2800330F8212002EA08021A4352
:101870007CE0D21A326224E0FA1A1F463262727891
:10188000012A15D0002A4FD1B0F850203CF8023080
:101890006FF39F232CF802308FB33E2F35D807F01B
:1018A00001033CF8025003EB570345EA832339E078
:1018B000B0F850202CF8027036E0002286F8242080
:1018C0002B467278012A15D0002A3FD1B0F850700B
:1018D0003CF807206FF39F222CF8072093B13E2B92
:1018E00025D803F001023CF8075002EB530245EA09
:1018F000822229E0B0F850202CF8023026E03CF893
:1019000002300DE03CF807201CE07B09FD063CF8A6
:1019100002E04FF0FF3508BF05EB57134EEA832373
:1019200043F400432CF802303289BBB210E05A096C
:10193000DD063CF807E04FF0FF3508BF05EB53121A
:101940004EEA822242F400422CF8072072899BB2B0
:1019500003F086FB2068317840F63F7330F8212091
:1019600048F2C0051A40A5F110035A4020F8212082
:10197000BCE42068B0F8441021F48061A0F8441061
:10198000204600F029FA94F89002012808D103B00B
:1019900000F08EB82068B0F8441021F4804133E0A4
:1019A0000120002584F8900265732068002103F06F
:1019B00043FB84F8905203B000F07AB82068B0F886
:1019C000441021F400511FE02068B0F8401021F0CD
:1019D0000401A0F84010B0F8401021F00801A0F870
:1019E000401094F8C802012806D1002084F8C802EB
:1019F00020460021FFF7AEFA204600F0FFF92068EC
:101A0000B0F8441021F48051A0F8441003B000F065
:101A10004FB82168B1F8400040F00800A1F840003C
:101A2000B1F8440020F40060A1F84400B1F840008F
:101A300040F004022046A1F840200AE02068B0F8F7
:101A4000441021F08001A0F8441094F8C81291B11C
:101A5000204603B000F02FB800F030BA2168B1F88A
:101A6000440020F400722046A1F8442003B000F0A6
:101A700027B800F0D7B9B0F8401041F00401A0F841
:101A80004010B0F8401041F00801A0F840100121CA
:101A900084F8C812B0F854003C2101EA90022046B4
:101AA0000121C4F8CC2203B000F00FB8FFF752BAFE
:101AB00030BCBDE8C08F30BCBDE8C04FFFF7CCBF25
:101AC00030BCBDE8C04FFFF7D4BF30BCBDE8C04F4D
:101AD000FFF7ECBF002804BF01207047F0B581B0CC
:101AE000044690F8910228B9002084F8900220461C
:101AF00000F02EF9032084F8910220680021617122
:101B000002F0B0FE94E80700237B02F019FE0028E3
:101B100040F0F2802068002103F08CFA002840F0A9
:101B2000EB8094F804E0BEF1000F00F0DF800EF0CF
:101B3000030CBEF1040F4FF0000237D30EF0FC038C
:101B4000A4F1A00003210125CE1E80F8B0608E1EF6
:101B500080F8D8604E1E80F8006180F828110E1DB4
:101B6000013180F8B15080F8B320C0E93022C0F8CC
:101B7000C82080F8D95080F8DB20C0E93A22C0F8AC
:101B8000F02080F8015180F80321C0E94422C0F818
:101B9000182180F8295180F82B21C0E94E22C0F885
:101BA0004021A03099423146CED1F21EBCF1000F47
:101BB0002ED004F1100002EB820100EBC1050123DD
:101BC00000F831200021BCF1010F6B70E970C5E90C
:101BD0000411A9611CD0551C05EB850600EBC60756
:101BE000BCF1020F7B7000F83650F970C7E90411A0
:101BF000B9610DD0911C01EB810200EBC2030125FC
:101C000000F8321000205D70D870C3E904009861BC
:101C1000BEF1000F6AD0BEF1040F4FF0000235D3C1
:101C20000EF0FC0003212346CF1E83F850718F1E57
:101C300083F878714F1E83F8C8110D1D013183F8A8
:101C4000512183F85321C3E95822C3F8682183F84E
:101C5000792183F87B21C3E96222C3F8902183F8BC
:101C6000A12183F8A07183F8A321C3E96C22C3F8F2
:101C7000B82183F8C92183F8CB21C3E97622C3F8C0
:101C8000E021A03381422946CED1EA1EBCF1000FEB
:101C90002CD004F5A87002EB820300EBC3070021EF
:101CA000BCF1010F797000F83320F970C7E9041115
:101CB000B9611BD0531C03EB830700EBC706BCF1D3
:101CC000020F717000F83730F170C6E90411B1618C
:101CD0000CD0911C01EB810200EBC20300275F7066
:101CE00000F83210DF70C3E904779F6194E80700C1
:101CF000237B02F0A9FD28B1022084F89102012083
:101D000001B0F0BD00206073012084F89102E07AF8
:101D1000012802D12046FFF707F9206802F08AFD6A
:101D2000002001B0F0BD0000006846F60001C4F2DA
:101D30000001884218BF704741F25801C4F2020105
:101D4000086820F0806243200A60FFF787B800002F
:101D500010B59AB0044602A820304021FEF713FBCC
:101D6000206846F60001C4F20001884201D01AB092
:101D700010BD4FF4005002904FF08060149003208B
:101D80000390012004900C2005900720069002206B
:101D9000CDE907004FF48010099002A800F0FAF88E
:101DA000002818BFFEF7DEFB41F25800C4F2020023
:101DB0000168002241F0806101600068002100F0AC
:101DC0008060019001984320FFF770F84320FFF7EF
:101DD0005BF81AB010BD000010B5044680790228E7
:101DE00018BFFEF7BFFBD4F8DC02012101F0D8FFD9
:101DF000D4F8DC02BDE8104001F088BF10B50446FD
:101E0000807A48B14EF61050CEF20000016821F001
:101E10000601016001F0A6F9D4F8DC02BDE810402B
:101E200001F0A4BFD0F8DC0201F0AABF90F8902224
:101E3000012A04BF0220704710B5012280F89022C9
:101E4000417302680446104603F0F6F8002084F857
:101E5000900210BDD0F8DC2200F52671104601F08A
:101E6000B5BF000090F89012012904BF022070470E
:101E700010B50168012280F890220446084603F05C
:101E80007DF8206802F0CCFC002084F8900210BDA0
:101E900090F89012012904BF0220704710B5016824
:101EA000012280F890220446084602F0DBFC2068FC
:101EB00002F0C0FC002084F8900210BD10B504466A
:101EC000D0F8DC0201F0E8FFA07A002808BF10BDBE
:101ED0004EF61050CEF20000016841F0060101609C
:101EE00010BD000047F20001C4F200010A68B0F51D
:101EF000007F02F4C06031D1B0F5007F2CD00868BB
:101F0000012262F34A20086040F22400C2F200007D
:101F10000068322250434DF68362C4F21B32A0FBAC
:101F20000202900C4A69520511D5421C0FD04A6931
:101F300052050CD558B14A69520508D5012806D07A
:101F40004A69520503D50228A0F10400EAD1486984
:101F5000400544BF0320704700207047B0F5806FF4
:101F6000FAD00868022262F34A2008600020704715
:101F700047F20400C4F20000016841F4806101608E
:101F80007047000047F20000C4F20000006800F44F
:101F9000C06070472DE9F04381B00446407841F2BB
:101FA00088070007C4F202071DD5606C78B1B0F550
:101FB000400F13D0B0F5000F40F0418157F87C0C72
:101FC00040F4803047F87C0C4FF4000006E0201D00
:101FD000002101F029F8814638B9606C396821F494
:101FE0004001084338604FF00009A078800750D5C1
:101FF00057F8300C5FEAC0080BD457F8300C40F0AB
:10200000805047F8300C57F8300C00F080500090AA
:10201000009847F20005C4F20005286840F480707B
:102020002860FEF7AFFE06462868C00507D4FEF715
:10203000A9FE801B0228F7D94FF0030920E0B9F16F
:10204000000F1DD1B86810F4407011D0E16D8842C6
:102050000BD0B868B96820F4407041F48031B960A1
:10206000B96821F48031B960B860C00740F0EA80F7
:10207000B868E16D20F4407008434FF00009B86083
:10208000B8F1000F05D457F8300C20F0805047F815
:10209000300C2168C80712D1880718D448071ED40D
:1020A000880624D488052AD4480530D4480636D476
:1020B00008063CD4C80542D4880448D459E038689E
:1020C000226A20F00300104338608807E6D538689C
:1020D000626A20F00C00104338604807E0D5386889
:1020E000A26A20F03000104338608806DAD53868DC
:1020F000E26A20F44060104338608805D4D538681F
:10210000E26B20F44020104338604805CED5386893
:10211000226C20F44010104338604806C8D5386857
:10212000226B20F44050104338600806C2D538684E
:10213000626B20F4404010433860C805BCD5386855
:10214000A26B20F4403010433860880411D53A68FF
:10215000A06C22F040620243B0F1806F3A601DD063
:10216000B0F1006F05D157F87C0C40F4801047F8AF
:102170007C0C080325D53A68E06C22F040620243EB
:10218000B0F1806F3A6014D0B0F1006F19D157F8F8
:102190007C0C40F4801047F87C0C12E0201D0121DB
:1021A00000F042FF2168002818BF81460803E2D4EE
:1021B00007E0201D012100F037FF2168002818BF2B
:1021C0008146480311D53A68206D22F040620243EF
:1021D000B0F1806F3A601CD0B0F1006F05D157F8B4
:1021E0007C0C40F4801047F87C0C48041BD5386800
:1021F000626D20F040501043B2F1805F386012D120
:10220000201D022100F010FF2168002818BF814620
:1022100009E0201D012100F007FF2168002818BFF8
:1022200081464804E3D4080405D53868A16D20F040
:10223000804008433860484601B0BDE8F0834FF065
:102240000109D2E6FEF79EFD064641F288354FF0C1
:10225000030900BFB86880073FF50AAFFEF792FD9B
:10226000801BA842F6D90BE72DE9F04381B0002886
:1022700000F0C48042F20009C4F202090446D9F811
:10228000000000F0070081420DD9D9F8000020F0CD
:1022900007000843C9F80000D9F8000000F0070063
:1022A000884240F0AB80206841F2080610F002023C
:1022B000C4F202060AD0A368376807F0F007BB42F1
:1022C00004D9376827F0F0073B433360C30733D0A6
:1022D000606856F8082C48B1022804D0032808D1B9
:1022E000920109D48AE0920306D487E0920703D4CE
:1022F00084E0520540F182808846316821F0030174
:1023000008433060FEF73EFD054641F2883700BFC6
:102310003068616800F00C00B0EB810F08D0FEF768
:1023200031FD401BB842F3D9032001B0BDE8F08372
:102330002068414600F0020252B1A268336803F0FF
:10234000F0039A4204D2336823F0F0031A43326058
:10235000D9F8002002F0070291420CD2D9F80020EF
:1023600022F007020A43C9F80020D9F8002002F041
:1023700007028A4242D1410705D53168E26821F45B
:10238000E06111433160000706D53068216920F40F
:10239000605040EAC10030603068716810F00C0095
:1023A00005D00C282ED101F0030101292AD156F8BD
:1023B000081C042211F008016FF0070108BF8C21EE
:1023C000715808BF0822D14045F6084201F00F01BC
:1023D000C0F6000252F8211000280A4618BF002259
:1023E0000C2838D1706800F00300022813D00328AD
:1023F00004BF41F20021C0F27A0110E0012001B0D7
:10240000BDE8F08304281DD0082820D141F2002225
:10241000C0F27A021FE042F20041C0F2F40170689B
:102420007268C0F30210C2F3062251437268013091
:10243000B1FBF0F0C2F34161022202EB4101B0FBBB
:10244000F1F208E042F20042C0F2F40203E000229E
:1024500000210C28C6D0306845F6EE31C0F30310D9
:10246000C0F60001085C00F01F0022FA00F140F203
:102470004010C2F2000040F224020068C2F20002E2
:10248000116001B0BDE8F043FEF7A0BC70B541F2A9
:102490000005C4F20205286840F001002860FEF73C
:1024A00071FC04462868800706D4FEF76BFC001B0D
:1024B0000228F7D9032070BD2868062161F30710B0
:1024C00028600020A86040F24010C2F2000040F2F4
:1024D0002401006840F60012C2F20001C0F23D0281
:1024E0000A60FEF773FC00281CBF012070BDFEF7D8
:1024F00049FC044641F28836A86810F00C0F06D05B
:10250000FEF740FC001BB042F6D9032070BD2868DE
:102510004FF2FF41CFF6FE2108402860FEF732FC63
:10252000044600BF286810F0206F06D0FEF72AFC92
:10253000001B0228F6D9032070BD0020E860E9687E
:1025400041F48051E9602861296941F48051296191
:10255000296821F4802129604FF0FF31A8612962A8
:10256000D5F8941041F40001C5F8941070BD000036
:1025700040F22400C2F200000068704740F22400DC
:1025800041F20801C2F20000C4F2020100680968C9
:1025900045F6FE32C1F30221C0F60002515C01F0A3
:1025A0001F01C8407047000040F2240041F20801BA
:1025B000C2F20000C4F202010068096845F6FE326A
:1025C000C1F3C221C0F60002515C01F01F01C840F6
:1025D0007047000041F20C01C4F2020151F8040CF2
:1025E00010F00C02086805D00C2A2BD100F0030073
:1025F000012827D151F80C0C042310F008006FF0CB
:102600000B0008BF8820085808BF0823D84045F6AB
:10261000084300F00F00C0F6000353F82030002AF2
:10262000184618BF00200C2A18BF7047086800F031
:10263000030002280FD0032804BF41F20023C0F298
:102640007A030CE0042A1DD0082A20D141F2002090
:10265000C0F27A00704742F20043C0F2F403086807
:102660000A68C0F30210C2F30622096801305A4317
:10267000B2FBF0F0C1F34161022202EB4101B0FB79
:10268000F1F0704742F20040C0F2F40070470020C1
:102690000023C8E7002804BF012070472DE9F0435C
:1026A00083B041F200060446C4F20206B068F16845
:1026B000227800F00C09D00601F003081CD4207821
:1026C000C00750D0B9F1080F46D0B9F10C0F08BFC0
:1026D000B8F1030F40D061683068B1F5803F07D092
:1026E000B1F5A02F40F03E8240F480203060306889
:1026F00040F4803030603FE2B9F1000F1CD0B9F1F6
:102700000C0F08BFB8F1010F16D0A169306800297D
:1027100000F08F8140F001003060FEF733FB05468A
:102720003068800700F19881FEF72CFB401B0228DF
:102730004FF00300F4D943E33068800703D5A06964
:10274000002800F0F582256A3068000700F10B814F
:10275000D6F89400000907E13068800303D560686B
:10276000002800F0E582207880072CD5B9F1040F0D
:102770001BD0B9F10C0F08BFB8F1020F15D0E168FA
:102780003068002900F0088240F480703060FEF765
:10279000F9FA0546306840050ED4FEF7F3FA401BFF
:1027A00002284FF00300F5D90AE33068400503D54D
:1027B000E068002800F0BC827068216920F0F850C1
:1027C00040EA016070602078000760D420784007FC
:1027D00074D42078800600F1AB80A06A002800F055
:1027E0004782022840F04A81F068E16A00F0030263
:1027F0008A4240F05B81226B6FF00F0300F07001A2
:1028000003EB0212914240F05181616B00F4FE42F1
:10281000B2EB012F40F04A81A16B00F07842B2EB9D
:10282000C16F40F04381E26B0023CFF6E07303EA0F
:10283000025200F4C001A2F50012914240F036812C
:10284000216C4FF07E4202EA016100F0C06001F1AC
:102850007E41884240F02A813068800100F1088280
:10286000306840F080703060F06840F08070F06058
:10287000FEF788FA04463068800100F1F981FEF71E
:1028800081FA001B02284FF00300F4D998E2616935
:10289000D6F89400002900F0B88040F00100C6F896
:1028A0009400FEF76FFA0546D6F8940080078DD4A1
:1028B000FEF768FA401B0228F6D94FE1B06D5FEAD7
:1028C000C00808D4B06D40F08050B065B06D00F025
:1028D00080500090009847F20007C4F20007386863
:1028E000C00512D4386840F480703860FEF74AFAA8
:1028F000054600BF3868C00507D4FEF743FA401B01
:1029000002284FF00300F5D95AE2A168D6F89000EA
:10291000012908D0052940F0068140F00400C6F8DE
:102920009000D6F8900040F00100C6F8900006E153
:10293000616AD6F89800002900F0E18040F00100BB
:10294000C6F89800FEF71EFA054600BFD6F89800B4
:1029500080073FF542AFFEF715FA401B02284FF003
:102960000300F3D92CE2306800F0F00085421BD957
:10297000B06DC00000F1B680B06D40F08050B06521
:10298000B06D00F0805001900198FFF7FBFAB16D37
:1029900021F08051B165B0F5007F00F0A980802D55
:1029A00040F20C81032013E13068B9F1000F40F0D0
:1029B00008003060306820F0F00040EA0500306028
:1029C0007068E16920F47F4040EA0120706040F0C7
:1029D0007B81B06DC00000F11C81B06D40F0805073
:1029E000B065B06D00F0805002900298FFF7CAFA0F
:1029F000B16D21F08051B165B0F5007F00F00F811D
:102A0000802D40F24981032050E120F00100C6F8FA
:102A10009400FEF7B7F90546D6F8940080077FF5D5
:102A2000D5AEFEF7AFF9401B02284FF00300F3D9F3
:102A3000C6E120F001003060FEF7A4F9054600BFB2
:102A4000306880077FF53BAEFEF79CF9401B0228FB
:102A50004FF00300F4D9B3E1306840F00800306073
:102A60003068D4E9071220F0F0001043306070683D
:102A700020F47F4040EA0120706020E6B9F10C0F9D
:102A800000F05681306820F080703060FEF77AF9EF
:102A9000044600BF3068800140F1E380FEF772F920
:102AA000001B02284FF00300F4D989E1B9F10C0FA3
:102AB00000F03E813068400100F13A81306820F03A
:102AC00080703060FEF75EF9054600BF3068800117
:102AD00040F17981FEF756F9401B02284FF00300C0
:102AE000F4D96DE1FFF74EFAB0F5007F7FF457AFF0
:102AF000812D6CD30120A02D88BF022068E020F03A
:102B00000100C6F89800FEF73DF90546D6F8980092
:102B100080077FF562AEFEF735F9401B02284FF0C3
:102B20000300F3D94CE120F00100C6F89000D6F87C
:102B30009000002920F00400C6F8900076D0FEF73F
:102B400021F9054641F28837D6F89000800700F158
:102B50007F80FEF717F9401BB842F5D9032003B078
:102B6000BDE8F08320F4803030603068002920F424
:102B70008020306000F08080FEF704F9054600BF39
:102B8000306880033FF5EFADFEF7FCF8401B64288A
:102B90004FF00300F4D913E120F480703060FEF7A9
:102BA000F1F80546306840057FF50DAEFEF7EAF80E
:102BB000401B02284FF00300F4D901E1A5F1700099
:102BC000B0FA80F04009802D08BF022000E000200C
:102BD00042F20001C4F202010A6822F00702024434
:102BE0000A60096801F00701814240F0A180306865
:102BF00040F0080030603068D4E9071220F0F0009F
:102C000010433060706820F47F4040EA012070601B
:102C10005AE0FFF7B7F9B0F5007F7FF4F1AE812DF0
:102C200043D30120A02D88BF02203FE0FEF7AAF881
:102C3000054641F2883700BFD6F89000800707D5D7
:102C4000FEF7A0F8401BB8424FF00300F4D9B7E0FC
:102C5000B8F1000F3FF5BDADB06D20F08050B0650C
:102C6000B7E5F0684FF6FC71CFF6EE610840F06012
:102C7000002003B0BDE8F083FEF784F8054600BFEE
:102C8000306880037FF56FADFEF77CF8401B642849
:102C90004FF00300F4D993E0A5F17000B0FA80F092
:102CA0004009802D08BF022000E0002042F2000110
:102CB000C4F202010A6822F0070202440A600968AD
:102CC00001F00701814233D1B068F16810F00C00C7
:102CD00005D00C2830D101F0030101292CD1314657
:102CE00051F8942B12F00802324608BF0A464FF002
:102CF0000401126808BF082122FA01F145F60842D2
:102D000001F00F01C0F6000252F8211000280A4617
:102D100018BF00220C2838D1F06800F00300022808
:102D200013D0032804BF41F20021C0F27A0110E061
:102D3000012003B0BDE8F08304281DD0082820D16D
:102D400041F20022C0F27A021FE042F20041C0F2DA
:102D5000F401F068F268C0F30210C2F30622514396
:102D6000F2680130B1FBF0F0C2F34161022202EBE4
:102D70004101B0FBF1F208E042F20042C0F2F4027D
:102D800003E0002200210C28C6D0B06845F6EE31E1
:102D9000C0F30310C0F60001085C00F01F0022FA27
:102DA00000F140F24010C2F2000040F2240200683C
:102DB000C2F200021160FEF709F800283FF47FAC70
:102DC00003B0BDE8F083F06848F28C01C0F29D11B9
:102DD00004F12C0700EA010C8ECF6FF00F00D4E94C
:102DE0000F5400EB02100022CFF6E07241EA0C0112
:102DF00002EA05520843A2F500124FF07E4540EA70
:102E0000032005EA0465104305F17E4540EAC760EA
:102E10002843F060306840F080703060F06840F027
:102E20008070F060FDF7AEFF0446306880013FF52A
:102E30001FAFFDF7A7FF001B02284FF00300F4D9D6
:102E4000BEE70000411E0020B0EB116F1CBF012047
:102E500070474EF21002CEF2000251604EF623513E
:102E6000CEF20001F0230B700721906011607047D3
:102E7000FEE70000F0B587B0002641F24C00069650
:102E8000CDE90466CDE90266C4F20200016840F2B1
:102E9000004441F0040101600168C4F6000401F03F
:102EA000040101910199016802AD41F080010160C6
:102EB0000168032701F0800101910199016841F047
:102EC00001010160016801F00101019101990168AE
:102ED00041F0020101600068294600F00200019003
:102EE00001984FF46040029004F58060CDE90376CC
:102EF000FDF766FE48F2FF70CDE902074FF0904003
:102F000029460496FDF75CFE4FF6FF70CDE90207F7
:102F1000204629460496FDF753FE0820CDE9020716
:102F200004F5C05029460496FDF74AFE07B0F0BDEF
:102F3000B0B586B0002441F24C000594CDE90344BD
:102F4000CDE90144C4F202000168002241F0010110
:102F5000016000684FF4805100F00100009000987B
:102F60004FF090404FF48055FDF706FF012002908E
:102F70000220CDE9030401A94FF090400195FDF72F
:102F80001FFE4FF090404FF480510022FDF7F4FEF9
:102F90004FF4FA70FDF756FC4FF090404FF480511B
:102FA0000122FDF7E9FE4FF4FA70FDF74BFC40F605
:102FB000F05040F20401C2F20000C2F2000100220F
:102FC00000F040FD002818BFFDF7CCFA40F6F050A5
:102FD00040F22801C2F20000C2F2000100F088FFB6
:102FE000002818BFFDF7BEFA40F6F05040F2D001BD
:102FF000C2F20000C2F2000100F0A8FA002818BFD7
:10300000FDF7B0FA40F6F050C2F2000000F09AFF6F
:10301000002818BFFDF7A6FA06B0B0BDFEE7000015
:10302000FEE7000070470000F0B581B041F20005F6
:10303000C4F20205EA68920713D0EA68036802F056
:1030400003029A424FF0010240F08580002B00F00D
:103050008280EA684368C2F3021201329A4222D0A7
:103060000DE00268032A0CD0022A05D0012A06D1FD
:103070002B689B0703D50BE02B685B0508D4012266
:1030800069E02B689B035CBF2B685FEA4333F6D58E
:10309000EB6847686FF00F0623F0730306EB071722
:1030A0003B431A43EA60064628680F4620F08060DA
:1030B0002860FDF767FE04462868000105D5FDF786
:1030C00061FE001B0228F7D93EE02969B06832464C
:1030D000012F4FEA002008D0BFB948F2FF03D268A1
:1030E000C0F2FF731940D2061BE048F2FF03CFF68F
:1030F000FF1303F1B463194012690023CFF6E073A4
:1031000003EA0252A2F500120BE048F2FF03CFF6E9
:10311000FF13526919404FF07E4303EA026202F145
:103120007E42084310432861286840F08060286090
:10313000FDF728FE044600BF2868000106D4FDF70D
:1031400021FE001B0228F7D9032204E0B069296997
:10315000002208432861104601B0F0BD704700000E
:10316000FDF716BE10B596B00020CDE90D00CDE9F3
:103170000B00CDE90900CDE907004FF40070FEF720
:10318000B1FE20B1EFF3108072B600BFFEE7012060
:10319000032405904FF48031CDE9104014200691AE
:1031A000022112900720CDE9130105A80F91159176
:1031B000FFF770FA18B1EFF3108072B6FEE70F2038
:1031C000CDE9000400204FF480610290CDE90310A6
:1031D00068460421FFF748F818B1EFF3108072B683
:1031E000FEE716B010BD00004EF68850CEF200008B
:1031F000016841F47001016070470000D0F8D422EA
:1032000000EB820CDCF8C032002B04BF03207047B7
:10321000B0B501F00F0202EB820400EB840E5EF801
:10322000182F4AB1D0F8C85205EBC404246AB2FB87
:10323000F4F505FB142292B10020C3F81402DCF867
:10324000C422D2F810C0BCF1000F08BFB0BDD3F843
:1032500008020A4603F50471E0470020B0BD0022D1
:103260000023CEF8002000F025FE0020B0BD0000B5
:10327000B0B5D0F8D42200EB8202D2F8C05295B19A
:10328000044600F0BDFCD4F8D412C5F80C0204EBDF
:103290008101D1F8C412D5F80402CA6805F503719A
:1032A00090470020B0BD0320B0BD000070B5812163
:1032B000044600F0EFFB002520460121258700F0A1
:1032C000E9FB20468221A4F8785100F0E3FBD4F812
:1032D000D402E56404F5307656F8201089B104EB89
:1032E0008000D0F8C40240688047D4F8D40256F871
:1032F000200001F09DF8D4F8D40246F82050C4F81C
:10330000BC52002070BD000010B5D0F8D41200EB04
:103310008100D0F8C04284B1D0F8C41259B194F8F9
:103320000002FF2807D08B6894F8012221469847B5
:10333000FF2084F80002002010BD032010BD000013
:10334000014640F2A4000A22C2F200000A8070473F
:10335000F0B581B040F26007C2F20007044638467B
:10336000822100F0B1FA06463846012100F0ACFA9D
:1033700005463846812100F0A7FA002E1CBF102117
:10338000B171002D1CBF4021A98000281CBF402125
:103390008180432140F26000C2F20000218001B030
:1033A000F0BD0000F0B581B040F26007C2F2000746
:1033B00004463846822100F087FA06463846012145
:1033C00000F082FA05463846812100F07DFA002E91
:1033D0001CBF1021B171002D1CBF4FF40071A980DA
:1033E00000281CBF4FF400718180432140F260002F
:1033F000C2F20000218001B0F0BD0000F0B581B044
:1034000040F26007C2F2000704463846822100F00D
:103410005BFA06463846012100F056FA0546384662
:10342000812100F051FA002E1CBF1021B171002D36
:103430001CBF4021A98000281CBF4021818043215E
:1034400040F26000C2F20000218001B0F0BD000037
:103450002DE9F04104464FF4077000F0EBFF00281F
:1034600050D04FF407710546FCF78DFFD4F8D40215
:10347000402704EB8000C0F8C052207CC4F8BC5246
:10348000002808BF4FF400772046812102223B46E6
:10349000022600F015FC4FF001082046012102220F
:1034A0003B46A4F8388000F00BFC1020A4F84E0036
:1034B0002046822103220823A4F8788100F000FC32
:1034C000D4F8D4020027C5F8047204EB8000D0F8C9
:1034D000C402A4F84C8000688047C5F81472C5F88F
:1034E0001872D5F8042252B1207C01210028204610
:1034F00014BF40234FF4007300F0F6FB0026304663
:10350000BDE8F081D4F8D402002104EB8000C0F8BB
:10351000C0120220BDE8F081D0F8D41200EB810186
:10352000D1F8C012002904BF0320704780B590F87D
:1035300010C0D1F8042240230121BCF1000F08BFC4
:103540004FF4007300F0D0FB002080BD00290FBFB6
:103550000320D0F8D42200EB8200C0F8C41218BFB8
:1035600000207047D0F8D42200EB8200D0F8C002CF
:1035700000280EBF0320C0F804120020704700008E
:10358000D0F8D43200EB8300D0F8C00200280FBF7F
:103590000320C0F80812C0F8102200207047000075
:1035A000F0B581B0D0F8D42200EB8203D3F8C0424A
:1035B0000022002C8DF80320ADF8002054D00D78A7
:1035C00015F0600214D0202A4CD1CA881AB36DB20B
:1035D000B5F1FF3F27DD4978402A84F800122146E3
:1035E00028BF402284F8012200F08EF800243CE03D
:1035F0004A780B2A36D80024DFE802F00637343444
:10360000343434343434253090F89C22032A29D1C0
:10361000694602221EE0D3F8C4020022836848787B
:103620000024984721E0D3F8C43206469D684B78C1
:103630000F4618462146A847FA883046072A28BF71
:103640000722214606E090F89C22032A0AD10DF1B8
:103650000301012200F072F8002406E090F89C2299
:10366000032A02D000F044F80324204601B0F0BD44
:10367000D0F8D41200EB8101D1F8C022002A04BF97
:1036800003207047D2F8141200294FF0010101D035
:103690000846704780B5C2F81412D2F81032D2F83A
:1036A00008228121C36200F005FC0021BDE88040B2
:1036B0000846704780B5D0F8B82252689047002875
:1036C00018BF032080BD0000002070470020704715
:1036D00080B513460A46002100F006FB002080BD9D
:1036E00080B513460A46002100F0E4FB002080BDAF
:1036F00010B58021044600F099FB20460021BDE86A
:10370000104000F093BB000080B513460A46032129
:10371000C0F894120021C0E9563300F0E5FA002009
:1037200080BD000080B50521C0F894120021002260
:10373000002300F0D9FA002080BD000080B51346B8
:103740000A460221C0F894120021C0E9063300F0B5
:10375000B1FB002080BD000080B50421C0F89412A8
:1037600000210022002300F0A5FB002080BD000006
:1037700010B5044600F07EFB012084F89C02D4F8CA
:10378000B80218B142682179204690470021C4F858
:10379000C412C4F8B4122046C4F8D012BDE81040D8
:1037A00000F01CBA10B540F2BC14C2F200040A4684
:1037B00002A0214600F0CAF8204610BD4344432031
:1037C000436F6E666967000040F2BC001222C2F2CD
:1037D00000000A807047000010B540F2BC14C2F22D
:1037E00000040A4602A0214600F0B0F8204610BDB1
:1037F00043444320496E746572666163650000004E
:1038000040F2E4000422C2F200000A807047000087
:1038100010B540F2BC14C2F200040A4602A02146D0
:1038200000F094F8204610BD53544D6963726F65E3
:103830006C656374726F6E696373000010B540F25B
:10384000BC14C2F200040A4602A0214600F07EF831
:10385000204610BD53544D33322056697274756141
:103860006C20436F6D506F72740000001A20088046
:1038700040F2E8003221C2F20000C0F23001C0F88C
:1038800002103821C0F23401C0F806103321C0F212
:103890003401C0F80A103621C0F23401C0F80E100D
:1038A0003521C0F23001C0F812103421C0F23701C6
:1038B000C0F816107047000040F2B0000C22C2F2AF
:1038C00000000A8070470000B0F802C003789C45F1
:1038D0009CBF0020704780B508E000BF82788A4214
:1038E00008BF80BD73449AB262452DD290F800E0C3
:1038F00070444278052A02D182788A4225D07344E6
:103900009AB2624520D290F800E070444278052ACD
:1039100002D182788A4218D073449AB2624513D297
:1039200090F800E070444278052A02D182788A42F9
:103930000BD073449AB2624506D290F800E070440E
:103940004278052ACAD0CDE7002080BD002808BFF4
:10395000704710B503783BB300F1020EF44600BF88
:103960001CF8013C5BB19CF8003043B19CF801307D
:103970002BB19CF802300CF1040C002BF0D14FF06D
:10398000000C00BF1EF8013C8BB19EF800308BB1DB
:103990009EF801308BB19EF802300CF1040C002B24
:1039A0000EF1040EEED10AE04FF0000C07E04CF0EF
:1039B000010C04E04CF0020C01E04CF0030C5FFA47
:1039C0008CFC022303EB4C03138003220B704A7020
:1039D00003789BB3023002224FF0000C5FFA82FEA4
:1039E00051FA82F401F80E3084F801C010F8013C5D
:1039F00023B3941C5FFA84FE51FA84F401F80E306C
:103A000084F801C00378CBB1141D5FFA84FE51FA2B
:103A100084F401F80E3084F801C0437873B1941D2A
:103A20005FFA84FE51FA84F401F80E3084F801C084
:103A300083780832002B00F10400CFD1BDE810409C
:103A400070470000002804BF032070470023C0F81F
:103A5000B832C0F8C4320029C0F8D03218BFC0F85C
:103A6000B412012180F89C12027000F0CDB8000061
:103A700080B5D0F8C802FDF70BFB40F20032C10060
:103A8000C0F2013222FA01F1032888BF0321C8B233
:103A900080BD000080B5D0F8C802FDF7D1FA40F231
:103AA0000032C100C0F2013222FA01F1032888BFBE
:103AB0000321C8B280BD0000B0B581B190F89C224E
:103AC000032A50D1D0F8B8225269002A4BD00023E3
:103AD000C0F8D4329047002808BF0020B0BDD0F80D
:103AE0009412022938D1D0E9071399420DD9CB1A83
:103AF00011461A46C3610446FFF7F2FD2046002135
:103B00000022002300F0F0F825E00FD182698A42FC
:103B10000CD3D0F898128A4208D200210022044621
:103B20000025FFF7DDFDC4F89852E7E790F89C12F6
:103B3000032909D1D0F8B812C96829B10022C0F808
:103B4000D4220446884720468021044600F06EF9BE
:103B50002046FFF7E7FD204690F8A01200291CBF81
:103B6000002180F8A0120020B0BD000010B579B18E
:103B700090F89C22032A1DD1D0F8B8229269CAB1CC
:103B80000023C0F8D4329047002808BF002010BDA1
:103B9000D0F8941203290DD1D0E9571399420BD9CB
:103BA000C91AC0F85C11994238BF0B4611461A4633
:103BB000FFF78EFD002010BD90F89C12032909D15B
:103BC000D0F8B812096929B10022C0F8D4220446FD
:103BD00088472046FFF7C0FD002010BD80B5D0F813
:103BE000C802FDF715FA40F20032C100C0F20132FE
:103BF00022FA01F1032888BF0321C8B280BD00006A
:103C0000D0F8C802FDF774BA10B50446FEF7B0F953
:103C100041F2D00046F60001C2F20000C4F20001F9
:103C20000160082101710221817101720021C0F837
:103C3000DC42C4F8C802C0F80910FDF74BFF0028A9
:103C400018BFFCF78FFCD4F8C8020021002218230B
:103C5000FDF7A8F9D4F8C802802100225823FDF707
:103C6000A1F9D4F8C80281210022C023FDF79AF9F6
:103C7000D4F8C802012100224FF48873FDF792F9AD
:103C8000D4F8C802822100224FF48073FDF78AF92C
:103C9000002010BDD0F8C80201F07F034AB203EB48
:103CA000830301EB810100EBC30300EBC10000F5CE
:103CB000A970002A48BF03F1120000787047000085
:103CC00080B59446D0F8C8021A466346FDF71AFA42
:103CD00040F20032C100C0F2013222FA01F10328A1
:103CE00088BF0321C8B280BD80B5D0F8C802FDF7F7
:103CF00039FA40F20032C100C0F2013222FA01F179
:103D0000032888BF0321C8B280BD0000F0B581B090
:103D10000126002580F89C62C0F894520446456054
:103D2000D0F8B802C4F8A45284F8A05240B1426856
:103D300032B12046002190470546002818BF0325D0
:103D400020460021002240234027FFF7B9FF2046EC
:103D5000802100224023A4F86461C4F86071FFF759
:103D6000AFFFA6842846276201B0F0BD90F89C12F0
:103D7000042904BF90F89D1280F89C12002070471F
:103D800090F89C12032908D1D0F8B81229B1C9695A
:103D900019B180B58847BDE8804000207047000019
:103DA000024600201174704780B5D0F8C802FEF7B3
:103DB0003DF840F20032C100C0F2013222FA01F1B6
:103DC000032888BF0321C8B280BD0000B0B500F24F
:103DD000AA240546204600F07FF80121C5F8941278
:103DE00095F8AA12B5F8B03201F01F02022AC5F800
:103DF00098320ED0012A06D08AB928462146BDE85D
:103E0000B04000F0A1B828462146BDE8B04000F01F
:103E1000D7BA28462146BDE8B04000F02FBA01F0DD
:103E200080012846BDE8B040AFF3008080B5D0F8EF
:103E3000C802FDF7B1F940F20032C100C0F2013210
:103E400022FA01F1032888BF0321C8B280BD000017
:103E500080B5D0F8C802FEF705F840F20032C10084
:103E6000C0F2013222FA01F1032888BF0321C8B24F
:103E700080BD000080B5D0F8C802FEF709F840F216
:103E80000032C100C0F2013222FA01F1032888BFDA
:103E90000321C8B280BD0000014690F89C020422B4
:103EA00004281CBF91F89C0281F89D02002081F833
:103EB0009C22704780B5D0F8C802FDF7A3F940F204
:103EC0000032C100C0F2013222FA01F1032888BF9A
:103ED0000321C8B280BD00000A7802704A7842709F
:103EE0004A8842808A888280C988C18070470000E1
:103EF00010B582B004460020ADF80600B1B1D4F888
:103F0000D42204F52E70C4F8B81250F82200C16A09
:103F100021B10DF106008847C4F8D002D4F8D802C8
:103F20000130C4F8D802002002B010BD032002B056
:103F300010BD0000D0F8B822002A04BF002070474E
:103F400012681047FFF784BF0A78C2F34112531E6C
:103F5000022B07D2D0F8D42200EB8202D2F8B8228A
:103F60009268104770B582B0002A40F0BE804A784F
:103F7000092A00F2BA80DFE802F0052CB84FB858E1
:103F800077B81A3C90F89C22013A022A00F2AD80E0
:103F9000C988022940F0A980D0F8A4120322002980
:103FA00008BF0122014641F80C2F022228E1C988EE
:103FB000012940F09A8090F89C124A1E022A80F053
:103FC0008F800024014641F8084F0122FFF7B6FB1D
:103FD00094E090F89C22013A022A00F286804988F7
:103FE0000024012940F08A80C0F8A442FFF7B4FB06
:103FF00084E0498840F2B815C2F2000511F0FE0FC6
:1040000029704BD080210446FFF710FF2046002185
:10401000FFF70CFF032471E04A88022A5CD0012AD2
:1040200063D10121C0F8A412EFE08A88002A5CD194
:10403000CA88002A59D14D887F2D56D890F89C12F5
:10404000032952D0E9B280F89E520446FFF7ACFE35
:1040500020462646FFF780FB002D14BF02200120DA
:1040600086F89C02002449E04A884FF0FF3303EBB6
:10407000122300260E2BADF8066000F27780DFE8F1
:1040800003F00858407575677375757575757575A6
:104090004C000D46D0F8B4120A6843E090F89C2218
:1040A000032A65D0022A40F087800A0600F0AD801E
:1040B00001F00102C9B242600546FFF73BFF00284C
:1040C00000F0BE80044628468021FFF7AFFE284658
:1040D0000021FFF7ABFE6BE0497980F8A01294E075
:1040E000032902D1011D01228AE080210446FFF745
:1040F0009DFE204600210024FFF798FE204602B0D6
:1041000070BDD2B2052A31D8DFE802F003AEA6AA0C
:10411000A2B2D0F8B422526802E0D0F8B422D26938
:1041200022B30D460446007C0DF10601904701467E
:104130005BE00D46017C0446D0F8B80200290CBFB4
:10414000816AC16A0DF106008847014602204BE0F2
:10415000027C5AB90446D0F8B8020D46416B0DF105
:1041600006008847014640E0027C9AB3044651E0CD
:104170000A0658D0426801F001018A4245D0D1B206
:104180000446FFF797FA2978204661602546FFF735
:10419000D1FE002870D0044628468021FFF746FE55
:1041A00028460021FFF742FE29792846FFF782FAC8
:1041B000022085F89C02A1E780210446FFF736FE25
:1041C00020460021FFF732FE29782046FFF772FAD9
:1041D000032493E70446D0F8B8020D46016B0DF1B5
:1041E00006008847014607204870EA8862B1BDF89A
:1041F000063073B1934238BF1A46ADF80620204608
:10420000FFF79CFA002479E72046FFF7A5FA00247F
:1042100074E720468021FFF709FE20460021FFF7C2
:1042200005FE00246AE7022180F89C120024002188
:1042300044600546FFF73EFA2846FFF78DFA5DE732
:104240002846FFF789FA032085F89C02002455E7E9
:10425000D0F8B422526963E7D0F8B422D2685FE79D
:10426000D0F8B42212695BE7D0F8B422926857E71D
:10427000D0F8B422926953E72846C6E770B50A78A9
:104280000D46C2F341120979531E022B044605D292
:104290002046FFF719FAD8B1002070BDE2BB68785C
:1042A00088B3012821D0032836D194F89C02032832
:1042B0001FD1688838B911F07F0004D0E88810B9A0
:1042C0002046FFF7B3FD2046FFF746FA002070BDF9
:1042D000D4F8B80282680020002AC4F8D402DBD0E7
:1042E00020462946BDE87040104794F89C020328F8
:1042F0001CD0022810D148060ED02046FFF796FDAC
:10430000204680210EE094F89C0203281ED002284B
:1043100008BF5FEA41603FD020468021FFF786FD5D
:1043200020460021FFF782FD002070BD688800282C
:10433000B2D10E46480603D020463146FFF798FB1F
:104340002046FFF709FA20463146A2E701F00F00A8
:1043500000EB8000802904EB80002CBF808CB0F83B
:1043600064010028D8D001F07F0000EB800004EB4E
:10437000800000F1140501EB810004EB800080292E
:1043800038BF00F5AA75480611D02046FFF782FC19
:10439000002818BF01200BE008064FF0140058BF9A
:1043A0004FF4AA70002221182250204603E000207A
:1043B0002860204629460222FFF7C0F9002070BD80
:1043C000B0B50A7802F06002602A08D090F89C220A
:1043D000013A022A03D88A8812F0FE0F0AD08021FF
:1043E0000446FFF723FD204600210024FFF71EFDB1
:1043F0002046B0BD0C46D1B20546FFF767F908B1BB
:104400000320B0BDD5F8B8128A68002AF8D0002180
:104410002846C5F8D41221469047E1880446002971
:1044200008BF002CE4D12846FFF796F90020B0BD64
:104430007047000040F2BC30C2F20000704700003C
:104440002DE9F0410B78024691F803E030F82300A3
:1044500047F27066BEF1030F20EA06040DD8002073
:10446000DFE80EF002050C0844F4007406E044F4A2
:10447000806403E044F4C06400E0012048F2800658
:10448000CFF6FF7644EA060522F8235032F823508F
:1044900040F60F7425401D432E4322F823600E7B07
:1044A00048F2800C002E52D032F8234040F60F65BF
:1044B0002C4048F28005BEF1020F08BF05F580755B
:1044C0002C4322F82340B2F850400E8902EBC3057A
:1044D0002C4426F00106A4F80064B2F850404E893E
:1044E0002C4426F00105A4F804544D7832F82340FA
:1044F000002D53D0610409D532F8231040F60F7413
:104500002140614401F5804122F8231032F8231044
:10451000490608D532F8231040F60F742140614453
:10452000403122F8231032F8231040F63F74214026
:104530000CF120044C40BEF1010F08BF41EA0C040D
:1045400022F8234032F8231043F60F77B9E04E7873
:10455000B2F85040CF88DD00002E27F001064DD084
:1045600051192144A1F8006432F82310490608D5F6
:1045700032F8231040F60F7421406144403122F894
:10458000231032F8231040F63F74BEF1010F01EA08
:10459000040100F097800CF12007CCE0670409D5F6
:1045A00032F8237040F60F763740674407F58047AE
:1045B00022F8237032F82370DD007F0608D532F828
:1045C000237040F60F7637406744403722F8237057
:1045D000B2F8504002EB050E0EF202452E5B6FF36F
:1045E0009F262E53096929B33E2925D801F00106DB
:1045F0002F5B06EB510647EA86262DE015442F195E
:10460000A7F80464B2F850E005F2064434F80E50FE
:104610006FF39F2524F80E500969002958D03E29D0
:1046200059D801F0010534F80E6005EB510146EA56
:10463000812161E0665B0AE0CF064FEA51162F5BED
:104640004FF0FF3808BF08EB511647EA862648F2BC
:104650000007CFF6FF773E432E53B2F850400EF2DC
:1046600006452F5B6FF39F272F5349B13E2909D889
:1046700001F001072E5B07EB510146EA812111E0B1
:10468000615B0AE0CE062E5B4FEA51174FF0FF3E0A
:1046900008BF0EEB511746EA872148F20007CFF614
:1046A000FF773943295332F8231043F60F77394007
:1046B0000CF54057794022F8231032F8231040F6C9
:1046C0003F77394041EA0C0122F82310BDE8F08120
:1046D0003EF804100BE0CF0634F80E704FEA511587
:1046E0004FF0FF3608BF06EB511547EA852148F227
:1046F0000005CFF6FF75294324F80E1032F8231079
:10470000490409D532F8231040F60F773940614447
:1047100001F5804122F823103BB132F8231043F613
:104720000F7739400CF5005705E0118843F60F77F5
:1047300039400CF54057794022F82310BDE8F0814C
:1047400000207047B0B50B7802460C7B487832F8F1
:1047500023104CF2800C002C4CF2800439D000283D
:1047600041D0480408D532F8230040F60F710840C4
:1047700040EA0C0022F8230032F8230043F60F7EB3
:10478000400640F63F7009D532F8231040F60F7509
:1047900029406144A1F57F5122F8231032F82310FB
:1047A00040F60F7529402143ACF5804422F82310D0
:1047B00032F823100840204322F8230032F8230067
:1047C00000EA0E006044A0F58041002022F823108A
:1047D000B0BDF0B1480640F63F7EEFD5ACF57F5452
:1047E00040F60F70E4E7480408D532F8230040F69D
:1047F0000F71084040EA0C0022F8230032F8230031
:10480000ACF57F54400640F63F7E43F60F70BBD4B4
:10481000C4E7480443F60F7ED0D540F60F70C7E7D3
:104820000146B0F8580040F400420020A1F858209A
:1048300070470000B0F8582001466FF3DF320020C7
:10484000A1F858207047000001460120A1F840005F
:1048500000220020A1F84020A1F84420A1F8502017
:10486000704700000146B0F8400044F27F02024069
:104870000020A1F8402070470020704791F800C048
:104880004A7830F82C30B2B15A0648F2A0030CD561
:1048900080B530F82CE040F60F7202EA0E021A449E
:1048A000203220F82C20BDE88040C978012918D09A
:1048B00040F63F710FE059044BF2800309D530F800
:1048C0002C1040F60F721140194401F5805120F868
:1048D0002C1043F60F7130F82C201140594020F86D
:1048E0002C1000207047000002460B78487832F800
:1048F00023C040F63F71002848F2900008BF43F6FD
:104900000F71CFF6FF7008BF00F57F6001EA0C0160
:104910004140002022F82310704700002DE9F04F9D
:1049200082B04A78012A5AD18B690A690F7B934277
:1049300028BF1346002F76D0CF780C6A022F40F0A4
:10494000AD800D7840F60F6630F825704FEA850E81
:10495000944206EA070648F2B00C40F2E38047F6BC
:104960005077F61BD036A4EB030A20F82560C1F877
:1049700020A030F82560B0F85070ED0076069EB2A9
:1049800000EB050800F1208108EB0704A4F80234CD
:10499000D1F814B0002E00F027820D8901360544AD
:1049A00005F580694FF0FF3505EB5604C6F3410568
:1049B000002D4FEA560700F08C815E46CDE9004895
:1049C00036F8028B5C46CB46012D2BF8028B40F06B
:1049D0008481DDF80480013FD946A346F2E10A7BD9
:1049E000002A48F2B00242D0CB78012B00F08A8036
:1049F000022B40F09380CF690B78002F00F0858068
:104A000030F8231044F240073940B94201D0002960
:104A10007BD130F8231040F60F7739401144103124
:104A200020F8231071E01A0400F02281CA88D1F81E
:104A300014E0024402F58068012212FA83F24FF07A
:104A4000FF37C2F3410407EB520C002C4FEA52022D
:104A500000F0FB80774637F8025B4646012C26F8CB
:104A6000025B40F0DA80013ABE46B046EDE08F6965
:104A70001FB9CB78002B00F0DC80A2F130060B7858
:104A800040F60F6430F8235025402E4320F8236071
:104A90000E69B74294BF0027BF1B35E0E21A0F78BA
:104AA0000A6230F82720B0F85040FD005206054455
:104AB0004FEA870E9AB248F2B00C2C4462D4002A16
:104AC000A4F8023400F0E0800B8901324969034404
:104AD0004FF0FF34C2F3410503F5806304EB520845
:104AE000002D4FEA520200F016810E4636F8024BB6
:104AF0001F46012D27F8024B40F0D380013A314682
:104B00003B4608E10B7800278F6142F6D0714FEAEF
:104B1000830E02EB010C43F60F71B7E0012002B0E7
:104B200000F029BA47F65072B21A303A20F8252020
:104B3000B0F8502000EBC5031A442304A2F8024445
:104B400000F0A2800A894969024402F580630122CB
:104B500012FA84F24FF0FF34C2F3410504EB52081D
:104B6000002D4FEA520200F0F1800E4636F8024B5B
:104B70001F46012D27F8024B40F09B80013A314639
:104B80003B46E3E0002AA4F806347DD04B8901328D
:104B9000496903444FF0FF34C2F3410503F58063D4
:104BA00004EB5208002D4FEA520200F0E9800E4655
:104BB00036F8024B1F46012D27F8024B40F081804A
:104BC000013A31463B46DBE008EB0705A5F8063421
:104BD000D1F814B0002E00F05D814D8901360544F6
:104BE00005F580694FF0FF3505EB5604C6F3410526
:104BF000002D4FEA56076ED05E46CDE9004836F8E4
:104C0000028B5C46CB46012D2BF8028B71D1DDF86F
:104C10000480013FD946A3462AE1BEF80250022C87
:104C2000A8F8025008D108F104080EF1040E023A67
:104C30000BE002F1D00622E7BEF804400EF1060EAA
:104C4000A8F8044008F10608033ABCF1030F0FD39B
:104C5000AEF10807A8F1080637F8085F043A26F80D
:104C6000085F7D887580BD88B580FD88F580F3D1AB
:104C7000B0F850200978024402EBC10248F2B00CAF
:104C8000A2F802344FEA810E40F63F7130F80E2050
:104C9000114081EA0C0120F80E10002002B000F053
:104CA0006AB94C88022D5C8030D104330431023A59
:104CB00031E04C88022D5C8043D104330431023A48
:104CC00044E04C88022D5C8055D104330431023A13
:104CD00056E05E4677E05E46CBE06688022DA3464E
:104CE000A9F8026063D109F104090BF10406023F3F
:104CF00066E06688022DA346A9F8026040F0AD8008
:104D000009F104090BF10406023FAFE08C8806317B
:104D10009C800633033AB8F1030FB5D3A1F1080420
:104D2000083B00BF34F8081F043A23F8081F6188C5
:104D30005980A1889980E188D98040F63F71F1D1EE
:104D4000A4E78C8806319C800633033AB8F1030F40
:104D50009AD3A1F10804083B34F8081F043A23F859
:104D6000081F61885980A1889980E188D98040F620
:104D70003F71F1D18AE78C8806319C800633033A73
:104D8000B8F1030FFFF480AFA1F10804083B00BFA6
:104D900034F8081F043A23F8081F61885980A18855
:104DA0009980E188D98040F63F71F1D16EE7BBF878
:104DB00004500BF10606A9F8045009F10609033F57
:104DC000DDF80480009C032C0ED3083EA9F10805F1
:104DD00036F8084F043F25F8084F74886C80B48873
:104DE000AC80F488EC80F3D10BEB030600244E6119
:104DF000924588BFAAEB03040C62B0F8502088BF2C
:104E00009A4608EB02031FFA8AF2002AA3F806A4C6
:104E10003FF43AAF4989013201444FF0FF33C2F306
:104E2000410401F5806103EB5208002C4FEA520265
:104E30006DD0354635F8023B0F46012C27F8023B72
:104E400003D1013A2E46394661E07388022C4B802B
:104E500058D104310436023A59E0BBF804500BF142
:104E60000606A9F8045009F10609033FDDF804809D
:104E7000009C032C0ED3083EA9F1080536F8084F14
:104E8000043F25F8084F74886C80B488AC80F4889F
:104E9000EC80F3D10BEB030600244E61924588BFF2
:104EA000AAEB03040C62B0F8502088BF9A4608EBC6
:104EB00002031FFA8AF2002AA3F802A43FF4E4AE28
:104EC0000989013201444FF0FF33C2F3410401F577
:104ED000806103EB52084FEA5202ACB3354635F815
:104EE000023B0F46012C27F8023B03D1013A2E4624
:104EF000394629E07388022C4B8020D104310436D6
:104F0000023A21E0B38806368B800631033AB8F1C5
:104F1000030FFFF4B9AEA6F10803A1F1080400BF26
:104F200033F8081F043A24F8081F598861809988CB
:104F3000A180D988E18040F63F71F1D1A6E6B3881F
:104F400006368B800631033AB8F1030FFFF49CAEAE
:104F5000A6F10803A1F1080433F8081F043A24F865
:104F6000081F598861809988A180D988E18040F61E
:104F70003F71F1D18AE630BCBDE8C08F0146002008
:104F80004BF68072A1F84400A1F840207047000061
:104F900041F2D000C2F20000FCF750B9B0F8440072
:104FA0007047000070B51044022B00F580643AD3BE
:104FB0004FF0FF32C3F34105580802EB530C4DB1DB
:104FC000224632F8026B8E46012D2EF8026B03D179
:104FD000013810E022460FE06288022D4A8004D199
:104FE000221D01F1040E023805E0A688A21D01F180
:104FF000060E03388E807146BCF1030F144613D39E
:1050000032F8086B043821F8086B32F8066C21F886
:10501000066C32F8046C21F8046C32F8026C21F84A
:10502000026CEDD114468E46D8071CBF20888EF83E
:10503000000070BD00207047002904BF8021A0F847
:105040004C1000207047000001460120A1F84000EC
:1050500000200322A1F84400A1F84020704700007E
:10506000002B08BF7047B0B5104400F5806E581C87
:105070004FF0FF32C0F3410302EB500C4FEA5000F7
:10508000BBB10A4632F8025B7446012B24F8025B7E
:1050900006D101381146A646BCF1030F0CD21BE025
:1050A0004A88022BAEF8022019D10EF1040E043109
:1050B0000238BCF1030F0FD30839AEF1080200BF6C
:1050C00031F8083F043822F8083F4B8853808B881A
:1050D0009380CB88D380F3D1BDE8B04070478A88F5
:1050E0000631AEF804200EF1060E0338BCF1030FB2
:1050F000E2D2F1E7FEE700004EF60C50BFF34F8F0F
:10510000CEF200000168042201F4E061C0F2FA521C
:1051100011430160BFF34F8F00BF00BF00BF00BF4E
:10512000FAE700002DE9F04385B0FBF731FD42F2CC
:10513000100048F29901C4F20200C0F201010160BE
:1051400041F2B030C2F20000006800F2FF70C117F7
:1051500000EB5150C11211F1100F07D3022000F0E3
:1051600005FD4FF41670FBF76DFBF7E7102101EB1F
:10517000E026102700244FF001090DF104086D46C8
:1051800002A8CDE9004480E89002EFF3108072B6E7
:1051900040462946FBF76AFB62B628B90137B74299
:1051A000EED905B0BDE8F083FBF708FC022000F063
:1051B000DDFC4FF41670FBF745FBF7E798B0FBF703
:1051C000F5FD0020CDE90F00CDE90D00CDE90B0084
:1051D000CDE909004FF40070FCF784FE18B1EFF33D
:1051E000108072B6FEE70120032407904FF480314F
:1051F000CDE9124014200891022114900720CDE936
:10520000150107A811911791FDF744FA18B1EFF3B2
:10521000108072B6FEE70F20CDE9020400204FF4A3
:1052200080610490CDE9051002A80421FDF71CF867
:1052300018B1EFF3108072B6FEE7FBF7A3FD40F65E
:10524000DC51C2F20001086010B90F20FBF7BEFD6F
:1052500048F20004C0F60004FDF70CFE4FF47A702B
:10526000FBF7F0FAFDF764FEFDF7B4F941F2F03117
:10527000C2F200010860FDF77BF941F2CC01C2F2F5
:1052800000010860FDF77AF941F2C831C2F200016D
:105290000860FDF789F941F2E132C2F200021278AA
:1052A00041F2CC31C2F20001012AA4F50064086089
:1052B0000CD100BF20460121FBF75AF918B1642038
:1052C000FBF7C0FAF6E76420FBF7BCFA40F2A81639
:1052D000C2F20006204631460822FBF78FF9D6E9D4
:1052E000000141F201025040084340F06F8201206A
:1052F0004FF0010A00F03AFC41F2F83041F2E83593
:1053000041F2EC3940F2000BC2F2000041F2E33707
:1053100041F2E43448F20006C2F20005C2F200098C
:105320004FF00008C2F2000B0830C2F20007C2F2D0
:105330000004C0F60006019005E000BF00F0E6FBA7
:10534000C82089F8000028780138032800F22A8252
:10535000DFE810F0040009017A00040141F2E930AD
:10536000C2F200000078012840D141F2E930C2F2D7
:10537000000080F8008041F2D030C2F20000A0F8B6
:10538000008041F2B430C2F20000A0F80080152085
:1053900089F8000040F6E050C2F20000C821017018
:1053A00041F2B630C2F20000A0F8008041F2D830DD
:1053B000C2F20000C0F8008041F2D430C2F2000016
:1053C000C0F8008041F2C030C2F20000C0F8008096
:1053D00041F2BC30C2F20000C0F8008041F2DC3083
:1053E000C2F20000CBF80060C0F8008041F2E23069
:1053F000C2F200000078012840F0D48140F23C1A4B
:10540000C2F2000A01248AF80080FFF78BFE8AF8B6
:10541000004041F2E83541F2E43441F2E3376420E0
:105420004FF0010AC2F20005C2F20004C2F2000706
:10543000FBF708FA0220287041F2E230C2F20000C5
:1054400080F80080AEE100BF3878012817D1152020
:1054500089F8000041F2B43040F6E051C2F2000099
:10546000C2F20001CA2200880A7041F2B631C2F2CB
:10547000000187F800800880FBF784FC2060FBF7C0
:1054800081FC2168401A40F2DD518842C0F08A81D7
:10549000002000F06BFBFBF791FA6420FBF7D2F9D8
:1054A00030680021C2F20201884251D83068B0F160
:1054B000005F4DD340F6F050C2F20000FEF758F9FD
:1054C0008AF31088FCF7E2FF4EF21000CEF20000E3
:1054D0004FF0FF31C0F80080C0F80480C0F80880A9
:1054E000C0F87011C0F87012C0F87411C0F87412CE
:1054F000C0F87811C0F87812C0F87C11C0F87C129E
:10550000C0F88011C0F88012C0F88411C0F884126D
:10551000C0F88811C0F88812C0F88C11C0F88C123D
:1055200048F2040088F31088C0F60000006840F2DA
:10553000B011C2F20001086040F2B411C2F20001E1
:105540000860306880F3088888F31488086880470A
:105550006420FBF777F90420287023E14FF41670DC
:10556000FBF770F91EE141F2EA30C2F20000007868
:10557000012840F0178141F2D030C2F20000B0F9AA
:10558000001041F2B430C2F20000B0F900004A1C31
:1055900082421AD141F2C630C2F2000090F800A057
:1055A0001AF0070745D0DBF80060BAF1080FC0F029
:1055B0009B8001994FEADA023046FBF7A1F80028F8
:1055C00000F08B80DBF800608EE080B289B2884208
:1055D00041F2EA31C2F2000181F8008013D140F2B9
:1055E0003C11C2F2000181F800A0152189F80010D9
:1055F00040F6E051C2F20001C92241F2C0330A7004
:10560000C2F200030CE0152189F8001040F6E051C9
:1056100041F2BC33C2F20001C922C2F200030A7097
:10562000196841F2B632C2F200021080481C1860BC
:10563000B8E0DBF8000001994FEADA02FBF760F806
:1056400041F2EA31002840F23C10C2F200014FF072
:10565000010AC2F2000081F8008080F800A007D0A3
:1056600041F2D431C2F2000108680130086027E03D
:1056700041F2D032C2F20002108840F6E851C2F284
:10568000000101300968108041F2B430CBF80010FD
:10569000C2F200001521008889F8001041F2B631ED
:1056A00041F2D832C2F20001C2F200020880106852
:1056B00040F6E051C2F20001C92301300B701060C6
:1056C00041F2E33741F2E43441F2E835C2F2000737
:1056D000C2F20004C2F2000564E040F6E850C2F2F3
:1056E00000000668CBF8006041F2F8310AF0F800DB
:1056F000C2F2000140F204140844C2F2000400F1B6
:10570000080120463A46FAF7D7FD304621460122E5
:10571000FAF7F6FF48F2000641F2E33741F2E434CB
:1057200041F2E835C0F600064FF0010AC2F2000768
:10573000C2F20004C2F20005A0BB41F2D031C2F2B5
:105740000001088841F2EA320130088040F6E85052
:10575000C2F20000006840F23C11C2F20001CBF836
:10576000000041F2B430C2F2000281F800A0C2F29F
:105770000000152182F80080008889F8001041F2AD
:10578000B63141F2D832C2F20001C2F20002088002
:10579000106840F6E051C2F20001C92301300B70DD
:1057A000106000BF99F8000015283FF4C7AD00282D
:1057B0007FF4C9AD4FF41670FBF744F84FF4167040
:1057C000FBF740F8012000F0D1F9BCE548F20005F4
:1057D000C0F6000528680021C2F6FE710840B0F14D
:1057E000005F4DD140F6F050C2F20000FDF7C0FF5F
:1057F000012080F31088FCF749FE4EF21001CEF232
:10580000000100204FF0FF32086048608860C1F856
:105810007021C1F87022C1F87421C1F87422C1F856
:105820007821C1F87822C1F87C21C1F87C22C1F826
:105830008021C1F88022C1F88421C1F88422C1F8F6
:105840008821C1F88822C1F88C21C1F88C2280F30C
:105850001088296848F20401C0F60001096840F286
:10586000B012C2F20002116040F2B412C2F20002A1
:105870001160296881F3088880F3148810688047D4
:105880004FF41670FAF7DEFF41F2B835C2F20005A8
:1058900007E000BFFBF792F8C820FAF7D3FFFBF749
:1058A00041FB4FF41670FAF7CDFF28780130C1B2F2
:1058B0000B292870F5D300BF20460121FAF758FEC6
:1058C0000028E7D06420FAF7BDFFF5E72DE9F041A5
:1058D00040F6EE56C2F2000640F6EC5296F8008012
:1058E000C2F20002157882F8008041F2F432C2F26E
:1058F000000241F2ED33147841F2EB31C2F20003C1
:10590000C2F2000141F2E03C1D700B78347040F6A9
:10591000ED56C2F2000CC2F200069CF80070137043
:105920003278012F0A7030703BD141F20451C2F23B
:1059300000010A6841F2F837C2F20007531CB8545C
:1059400040F21212C2F2000240F20C165078927825
:10595000C2F2000674788518C5F58577A74205EB75
:1059600004070B60BEBF00238CF800300B60BB4205
:1059700047D3204441F2F8340023C2F200040B6004
:10598000811820468CF80030FAF7F8FE002848D03D
:1059900040F6E450C2F20000016801310160BDE848
:1059A000F08140F20C1EC2F2000E9EF800108D42F3
:1059B00023D19EF803108B421FD19EF804108A4217
:1059C0001BD101218CF8001041F2F831C2F2000124
:1059D0008EF80500487141F204500D7081F8018085
:1059E0008C70CB700A71C2F2000006218EF8018023
:1059F0008EF802400160BDE8F081442808BF242CE5
:105A000001D0BDE8F081412BFBD1492A18BFBDE888
:105A1000F08141F2E130C2F2000001210170BDE8E5
:105A2000F0817079CA283ED0C92815D0C828E8D19D
:105A3000D4F8060041F2B031C2F20001086041F230
:105A4000E830C2F200000121017041F2E930C2F2F7
:105A500000000170BDE8F08141F2E830C2F20000C0
:105A60000078012843D00228CBD141F2EA30C2F2BB
:105A7000000001780029C4D140F23C11C2F20001BB
:105A800000220A7001210170E08841F2B431C2F2B3
:105A900000017278088041F2C631901EC2F2000106
:105AA0000870BDE8F08141F2B031C2F2000109682E
:105AB00048F68902C8F6880241F2D03052FB011143
:105AC000C2F20000B0F90000CA1102EBD1718142AC
:105AD00097DC41F2E830C2F200000178022904BFED
:105AE0000321017041F2E330C2F2000095E7E08843
:105AF00041F2B431C2F20001012808807FF481AF85
:105B000041F2E230C2F2000087E7000010B540F237
:105B10001210C2F2000041F2085401784279B0F844
:105B20000300C2F20004A4F803001520607140F6DF
:105B3000E0502170C2F2000041F2B6310078C2F2AA
:105B400000010988A0710320A4F8071060702046A6
:105B50000921A270FAF712FE024620460B21A4F892
:105B60000920BDE81040FAF7DFBC000070B541F233
:105B70000854C2F200040546E01D40F20311FAF792
:105B8000E0FB40F21210C2F2000001784279B0F856
:105B9000030041F2C436A4F80300C7206071C2F2CA
:105BA0000006072030800120217060702046072108
:105BB000A270A571FAF7E2FD3188030A4A1C60540D
:105BC000881C92B2308081B22046A354BDE8704058
:105BD000FAF7AABCF1EE100A4FF6FF71C0F2C0311D
:105BE00020EA010040F04070E1EE100A704700002A
:105BF000000000000000010203040607080900007D
:105C00000000010203040000A0860100400D030013
:105C1000801A060000350C0040420F0080841E00F0
:105C200000093D0000127A000024F40000366E01E5
:105C30000048E801006CDC0200C1814001C08041E5
:105C400001C0804100C1814001C0804100C181404C
:105C500000C1814001C0804101C0804100C181403C
:105C600000C1814001C0804100C1814001C080412C
:105C700001C0804100C1814001C0804100C181401C
:105C800000C1814001C0804100C1814001C080410C
:105C900001C0804100C1814000C1814001C08041FC
:105CA00001C0804100C1814001C0804100C18140EC
:105CB00000C1814001C0804101C0804100C18140DC
:105CC00000C1814001C0804100C1814001C08041CC
:105CD00001C0804100C1814000C1814001C08041BC
:105CE00001C0804100C1814001C0804100C18140AC
:105CF00000C1814001C0804100C1814001C080419C
:105D000001C0804100C1814001C0804100C181408B
:105D100000C1814001C0804101C0804100C181407B
:105D200000C1814001C0804100C1814001C080416B
:105D300001C0804100C1814000C0C101C30302C253
:105D4000C60607C705C5C404CC0C0DCD0FCFCE0EBB
:105D50000ACACB0BC90908C8D81819D91BDBDA1A2B
:105D60001EDEDF1FDD1D1CDC14D4D515D71716D69B
:105D7000D21213D311D1D010F03031F133F3F2320B
:105D800036F6F737F53534F43CFCFD3DFF3F3EFE7B
:105D9000FA3A3BFB39F9F83828E8E929EB2B2AEAEB
:105DA000EE2E2FEF2DEDEC2CE42425E527E7E6265B
:105DB00022E2E323E12120E0A06061A163A3A262CB
:105DC00066A6A767A56564A46CACAD6DAF6F6EAE3B
:105DD000AA6A6BAB69A9A86878B8B979BB7B7ABAAB
:105DE000BE7E7FBF7DBDBC7CB47475B577B7B6761B
:105DF00072B2B373B17170B050909151935352928B
:105E000096565797559594549C5C5D9D5F9F9E5EFA
:105E10005A9A9B5B99595898884849894B8B8A4A6A
:105E20004E8E8F4F8D4D4C8C4484854587474686DA
:105E30008242438341818040585E00080000002078
:105E400048010000F0010008405F00084801002000
:105E5000D01A0000300200082F00800008C9370067
:105E6000080138000811382C083D3800086D38004A
:105E700008A5372D08D9370008B938000800093DB2
:105E80005D51340008AD320008A1350008DD09334A
:105E90000008FD310008713200082FA533000851B9
:105EA000330008FD33000841333D08090243000276
:105EB0000100C03209042E01020201000524001075
:105EC000010524012901042402020524064F0107CB
:105ED00005820308001009040100020A36070501C3
:105EE0000240460705810240450A06000243400180
:105EF0004A050F0C0001071002022D1201010202D7
:105F0000020040830440573602010203012FC104FE
:105F10000008BD040008B9040008ED040C1B0825A6
:105F2000050008040309041A0382FF42FE0618054F
:105F300000FE060202100133010182100000000081
:040000050800018D61
:00000001FF
